:100000000200713200000000000000320000000019
:10001000000000320000000000000032000000007C
:10002000000000320000000000000032000000006C
:10003000000000320000000000000000000000008E
:10004000000000320000740D120051740A120051B9
:10005000223099FDC299F5992278617903D8FED9A9
:10006000FCD5E0F522E62401F6FA08E63400F64A6B
:100070002278FFE4F6D8FD758127C28E75985275F7
:100080008922438780758DFCD28E752000D2B0D234
:10009000B1752200120185752200120190120046EE
:1000A000780BE88360061200510880F60200DC201D
:1000B00020436F6E74656767696F2062696E617255
:1000C000696F20737569203136204C454473206474
:1000D000656C6C612054494F20313600120046781F
:1000E0000BE88360061200510880F60201314D6F63
:1000F0006E74617265204D696E69204D6F64756C18
:100100006F207375205A322064656C6C6120474DF6
:100110004D2054535433206520636F6C6C656761C8
:1001200072652054494F203136206120434E342ED1
:1001300000120046780BE88360061200510880F632
:10014000020158436F6E74656767696F20696E209E
:10015000636F72736F2E2E00752400752500E524E1
:10016000F5236323FF12018C782408E6F52363232B
:10017000FF12019D782412006574321200590201A9
:100180005EC2AF80FE7590FF85902322852390226A
:1001900043B0FC85B02343C00385C0232275F00122
:1001A000E52355F0C0E07826D0E0F6E526B400025D
:1001B00080030201BAC2B20201BCD2B275F002E5FC
:1001C0002355F0C0E07826D0E0F6E526B4000280A2
:1001D000030201D9C2B30201DBD2B375F004E523F7
:1001E00055F0C0E07826D0E0F6E526B400028003A2
:1001F0000201F8C2B40201FAD2B475F008E5235541
:10020000F0C0E07826D0E0F6E526B40002800302D4
:100210000217C2B5020219D2B575F010E52355F0E8
:10022000C0E07826D0E0F6E526B4000280030202A2
:1002300036C2B6020238D2B675F020E52355F0C0BA
:10024000E07826D0E0F6E526B400028003020255ED
:10025000C2B7020257D2B775F040E52355F0C0E0AF
:100260007826D0E0F6E526B400028003020274C2CC
:10027000C0020276D2C075F080E52355F0C0E07868
:1002800026D0E0F6E526B400028003020293C2C144
:10029000020295D2C1220000000000000000000010
:00000001FF
